:10027700454D4245444445442053595354454D53F5
:010287000076
:05029C00011E00C1027B
:0300030002026294
:10026200C0E0C0D0051EE51EB40403751E00D20214
:05027200D0D0D0E03205
:1000FC00E4F508F509F50AF50BC200780C7C00FD57
:10010C007BFF7A027977FE7F111200D6E4F59075A9
:10011C00B0FFF580120248D28875A881E4F508F585
:10012C0009740C2509F8E6FF600D1202880509E533
:10013C000970EE050880EA300220120248E4F50846
:10014C00F509740C2509F8E6FF600D120288050903
:10015C00E50970EE050880EAC202E51E640170280C
:10016C003000097F08120000C20080077F0C1200CB
:10017C0000D2007F647E001202287F1C1200007FD8
:0F018C00647E0012022880AFE51EB403AA80A88B
:01019B002241
:0E0288008F1D1202A2851D80D2011202962245
:06029600300102D2A0229B
:10022800E4FDFCC3ED9FEC9E5015E4FAFB0BBB000C
:0F023800010ABA01F8BB62F50DBD00010C80E4AC
:010247002294
:100248007F381200007F0C1200007F011200007F2F
:0A025800061200007F801200002251
:0102A2002239
:0300000002019C5E
:0C019C00787FE4F6D8FD7581200201E3B5
:10000600E709F608DFFA8046E709F208DFFA803EDC
:1000160088828C83E709F0A3DFFA8032E309F608C9
:10002600DFFA8078E309F208DFFA807088828C8331
:10003600E309F0A3DFFA806489828A83E0A3F608E5
:10004600DFFA805889828A83E0A3F208DFFA804CBF
:1000560080D280FA80C680D4806980F28033801096
:1000660080A680EA809A80A880DA80E280CA8033FF
:1000760089828A83ECFAE493A3C8C582C8CCC58377
:10008600CCF0A3C8C582C8CCC583CCDFE9DEE78047
:100096000D89828A83E493A3F608DFF9ECFAA9F0C6
:1000A600EDFB2289828A83ECFAE0A3C8C582C8CC1C
:1000B600C583CCF0A3C8C582C8CCC583CCDFEADE35
:1000C600E880DB89828A83E493A3F208DFF980CC97
:1000D60088F0EF60010E4E60C388F0ED2402B40490
:1000E6000050B9F582EB2402B4040050AF23234537
:0600F60082239000567306
:1001A8000200FCE493A3F8E493A34003F68001F271
:1001B80008DFF48029E493A3F85407240CC8C33358
:1001C800C4540F4420C8834004F456800146F6DF27
:1001D800E4800B010204081020408090029CE47E19
:1001E800019360BCA3FF543F30E509541FFEE4931C
:1001F800A360010ECF54C025E060A840B8E493A3E3
:10020800FAE493A3F8E493A3C8C582C8CAC583CA0D
:10021800F0A3C8C582C8CAC583CADFE9DEE780BEC5
:0102A100005C
:00000001FF
